:100000000C9435000C945D000C945D000C945D0024
:100010000C945D000C945D000C945D000C945D00EC
:100020000C945D000C945D000C945D000C945D00DC
:100030000C945D000C945D000C945D000C945D00CC
:100040000C94F9030C945D000C94A2020C94E5024C
:100050000C945D000C945D000C945D000C945D00AC
:100060000C945D000C945D00A30311241FBECFEF20
:10007000D8E0DEBFCDBF11E0A0E0B1E0E0E5F9E0FF
:1000800002C005900D92AE34B107D9F712E0AEE48C
:10009000B1E001C01D92A130B107E1F710E0CAE65E
:1000A000D0E004C02297FE010E94A204C836D10706
:1000B000C9F70E94FD010C94A6040C94000040E8CE
:1000C00055E260E070E08EE491E00E9420038EE44F
:1000D00091E00E94A1038823D1F362E071E08EE4F5
:1000E00091E00C942801E0914E01F0914F010190B4
:1000F000F081E02D609100018EE491E009956EE1C0
:1001000071E08EE491E00E940B016091000170911A
:1001100001014AE050E08EE491E00E94DD0166E2D8
:1001200071E08EE491E00E940B01609100017091FA
:10013000010140E150E08EE491E00E94DD016EE2B9
:1001400071E08EE491E00E940B01609100017091DA
:10015000010148E050E08EE491E00E94DD0166E399
:1001600071E08EE491E00E940B01609100017091BA
:10017000010142E050E08EE491E00E94E5018091AF
:100180000001909101018E37910509F4FFCF01968E
:1001900090930101809300010895CF92DF92EF9236
:1001A000FF920F931F93CF93DF936C017A01EB01C2
:1001B000E60EF71E00E010E0CE15DF0561F0699154
:1001C000D601ED91FC910190F081E02DC6010995D9
:1001D000080F191FF1CFC801DF91CF911F910F9127
:1001E000FF90EF90DF90CF9008956115710581F039
:1001F000DB010D900020E9F7AD0141505109461B8C
:10020000570BDC01ED91FC910280F381E02D099404
:1002100080E090E008950C94F500DC01ED91FC91F4
:100220000190F081E02D09940F931F93CF93DF93FA
:10023000EC016DE00E940D018C016AE0CE010E948C
:100240000D01800F911FDF91CF911F910F910895A4
:100250000F931F93CF93DF93EC010E94F5008C0165
:10026000CE010E941401800F911FDF91CF911F9149
:100270000F9108958F929F92AF92BF92CF92DF928B
:10028000EF92FF920F931F93CF93DF93CDB7DEB71B
:10029000A1970FB6F894DEBF0FBECDBF7C01C42E70
:1002A000E52FCB01D22E19A221E02D1510F02AE066
:1002B000D22E8E010F5D1F4F8D2C912CA12CB12CB5
:1002C0006C2D7E2FA50194010E947E048C2DD29E60
:1002D00080191124015011098A3014F4805D01C085
:1002E000895CF8018083211531054105510521F014
:1002F000C22EE32FCA01E4CFB801C7010E94F50066
:10030000A1960FB6F894DEBF0FBECDBFDF91CF919F
:100310001F910F91FF90EF90DF90CF90BF90AF9023
:100320009F908F900895CF92DF92EF92FF920F935C
:100330001F93CF93DF93EC016A017B0121153105F7
:1003400079F4E881F9810190F081E02D642FDF914B
:10035000CF911F910F91FF90EF90DF90CF90099474
:100360002A303105E9F477FF1AC06DE20E940D01D1
:100370008C0144275527BA014C195D096E097F0984
:100380002AE0CE010E943A01800F911FDF91CF91A8
:100390001F910F91FF90EF90DF90CF9008952AE08A
:1003A000B701A601CE01DF91CF911F910F91FF9070
:1003B000EF90DF90CF900C943A019A01AB01662741
:1003C00057FD6095762F0C9493010F931F93CF9355
:1003D000DF93EC019A01AB01662757FD6095762FFC
:1003E0000E9493018C01CE010E941401800F911F85
:1003F000DF91CF911F910F9108950E9443040E94B5
:100400005F00CCEDD2E00E9473002097E1F30E94E0
:10041000DC02F9CFFC0124853585F901E05CFF4F52
:1004200080819181F901EE5BFF4F20813181821B38
:10043000930B8F7399270895FC0184859585FC01A2
:10044000E05CFF4F40815181FC01EE5BFF4F20815A
:1004500031814217530741F00190F081E02DE80F00
:10046000F91F808190E008958FEF9FEF0895FC01C0
:1004700084859585FC01E05CFF4F40815181FC0142
:10048000EE5BFF4F208131814217530779F0A08145
:10049000B181A80FB91F8C91208131812F5F3F4F0F
:1004A0002F7333273183208390E008958FEF9FEFE0
:1004B0000895FC0181A1882329F0A489B5898C9134
:1004C00086FFFBCF11A20895CF93DF93FC01268511
:1004D0003785D901A05CBF4F8D919C9111970196F2
:1004E0008F739927E901CE5BDF4F488159818417CB
:1004F0009507D9F30D90BC91A02DA20FB31F6C935B
:10050000A685B785A05CBF4F11969C938E93A68954
:10051000B7892C9181E090E0078C02C0880F991F69
:100520000A94E2F7282B2C9381E081A30488F589B3
:10053000E02D80818064808381E090E0DF91CF9125
:10054000089508951F920F920FB60F9211242F93C2
:100550003F934F938F939F93EF93FF938091C000AE
:1005600082FD1CC04091C6008091F4019091F5017C
:1005700001968F7399272091F6013091F701821728
:10058000930771F0E091F401F091F501EC54FE4F06
:1005900040839093F5018093F40102C08091C600DE
:1005A000FF91EF919F918F914F913F912F910F90DC
:1005B0000FBE0F901F9018958EE491E00E940A02E2
:1005C000892B11F00C94A10208951F920F920FB67F
:1005D0000F9211242F933F938F939F93EF93FF9349
:1005E0002091B0013091B1018091B2019091B3019D
:1005F0002817390731F48091C1008F7D8093C100A5
:1006000014C0E091B201F091B301E059FE4F208196
:100610008091B2019091B30101968F7399279093C5
:10062000B3018093B2012093C600FF91EF919F9197
:100630008F913F912F910F900FBE0F901F901895A3
:10064000CF92DF92EF92FF92CF93DF93EC016A019A
:100650007B01411581EE580761057105F9F0EC89C0
:10066000FD8981E090E008A002C0880F991F0A94DC
:10067000E2F7808360E079E08DE390E0A7019601E6
:100680000E947E0421503109410951095695479530
:1006900037952795211580E1380798F0EC89FD8979
:1006A000108260E874E88EE190E0A70196010E9454
:1006B0007E042150310941095109569547953795D6
:1006C0002795E889F9893083EA89FB89208319A273
:1006D000EE89FF89408181E090E09C010C8C02C092
:1006E000220F331F0A94E2F7422B4083EE89FF89E1
:1006F00040819C010D8C02C0220F331F0A94E2F747
:10070000422B4083EE89FF8940819C010E8C02C000
:10071000220F331F0A94E2F7422B4083EE89FF89B0
:1007200020810F8C02C0880F991F0A94E2F78095F0
:1007300082238083DF91CF91FF90EF90DF90CF9065
:10074000089581E00895109251011092500188EEB1
:1007500093E0A0E0B0E08093520190935301A09306
:100760005401B093550182E491E090934F0180933E
:100770004E0184EB91E090935B0180935A0180E7F6
:1007800091E090935D0180935C0185EC90E0909303
:100790005F0180935E0184EC90E09093610180930F
:1007A000600180EC90E0909363018093620181ECA2
:1007B00090E0909365018093640182EC90E09093C7
:1007C00067018093660186EC90E0909369018093C5
:1007D000680184E080936A0183E080936B0187E085
:1007E00080936C0185E080936D0181E080936E01C0
:1007F00008951F920F920FB60F9211242F933F93DB
:100800008F939F93AF93BF938091F9019091FA01D9
:10081000A091FB01B091FC013091F80123E0230F7E
:100820002D3720F40196A11DB11D05C026E8230F28
:100830000296A11DB11D2093F8018093F9019093B8
:10084000FA01A093FB01B093FC018091FD0190910E
:10085000FE01A091FF01B09100020196A11DB11D02
:100860008093FD019093FE01A093FF01B0930002DD
:10087000BF91AF919F918F913F912F910F900FBE9C
:100880000F901F901895789484B5826084BD84B5CC
:10089000816084BD85B5826085BD85B5816085BD7B
:1008A000EEE6F0E0808181608083E1E8F0E0108294
:1008B000808182608083808181608083E0E8F0E0D5
:1008C000808181608083E1EBF0E0808184608083BF
:1008D000E0EBF0E0808181608083EAE7F0E08081F6
:1008E0008460808380818260808380818160808356
:1008F0008081806880831092C1000895A1E21A2E41
:10090000AA1BBB1BFD010DC0AA1FBB1FEE1FFF1FB3
:10091000A217B307E407F50720F0A21BB30BE40B03
:10092000F50B661F771F881F991F1A9469F760954A
:100930007095809590959B01AC01BD01CF01089504
:10094000EE0FFF1F0590F491E02D0994F894FFCF6E
:1009500021004153434949205461626C65207E2047
:10096000436861726163746572204D6170002C2070
:100970006465633A20002C206865783A20002C20BA
:100980006F63743A20002C2062696E3A20000000E8
:0E09900000006402CD000A0237021C02590268
:00000001FF
